:020000040000FA
:1000000000500400000000000CA20000E4A1000069
:10001000EAA10000F0A10000F6A100000CA200007F
:100020000CA200000CA200000CA200002E8900000F
:100030000CA20000AA8400000CA200000CA2000088
:100040000CA200000CA200000CA200000CA20000F8
:100050000CA20000D47C00000CA200000CA2000046
:100060000CA200000CA200006A6B00000CA20000B1
:100070000CA200000CA200000CA200000CA20000C8
:100080000CA200000CA200000CA200000CA20000B8
:100090000CA200000CA200000CA200000CA20000A8
:1000A0000CA200000CA200000CA200000CA2000098
:1000B0000CA200000CA200000CA200000CA2000088
:1000C0000CA200000CA200000CA200000CA2000078
:1000D0000CA200000CA200000CA200000CA2000068
:1000E0000CA200000CA200000CA200000CA2000058
:1000F000887500000CA200000CA200000CA20000F9
:100100000CA200000CA200000CA200000CA2000037
:100110000CA200000CA200000CA200000CA2000027
:100120000CA200000CA200000CA200000CA2000017
:100130000CA200000CA200000CA200000CA2000007
:100140000CA200000CA200000CA200000CA20000F7
:100150000CA200000CA200000CA200000CA20000E7
:100160000CA200000CA200000CA200000CA20000D7
:100170000CA200000CA200000CA200000CA20000C7
:100180000CA200000CA200000CA200000CA20000B7
:100190000CA200000CA200000CA200000CA20000A7
:1001A0000CA200000CA200000CA200000CA2000097
:1001B0000CA200000CA200000CA200000CA2000087
:1001C0000CA200000CA200000CA200000CA2000077
:1001D0000CA200000CA200000CA200000CA2000067
:1001E000FE900000589400000CA20000D087000090
:1001F000629D0000388D00000CA200000CA20000DF
:10020000FFFFFF00FFFFFF000C460000FC45000061
:100210000046000004460000084600000C460000AE
:100220000C4600000C4600000C4600002E2D00007D
:100230000C460000AA2800000C4600000C460000F6
:100240000C4600000C4600000C4600000C46000066
:100250000C460000D42000000C4600000C460000B4
:100260000C4600000C4600006A0F00000C4600001F
:100270000C4600000C4600000C4600000C46000036
:100280000C4600000C4600000C4600000C46000026
:100290000C4600000C4600000C4600000C46000016
:1002A0000C4600000C4600000C4600000C46000006
:1002B0000C4600000C4600000C4600000C460000F6
:1002C0000C4600000C4600000C4600000C460000E6
:1002D0000C4600000C4600000C4600000C460000D6
:1002E0000C4600000C4600000C4600000C460000C6
:1002F000881900000C4600000C4600000C46000067
:100300000C4600000C4600000C4600000C460000A5
:100310000C4600000C4600000C4600000C46000095
:100320000C4600000C4600000C4600000C46000085
:100330000C4600000C4600000C4600000C46000075
:100340000C4600000C4600000C4600000C46000065
:100350000C4600000C4600000C4600000C46000055
:100360000C4600000C4600000C4600000C46000045
:100370000C4600000C4600000C4600000C46000035
:100380000C4600000C4600000C4600000C46000025
:100390000C4600000C4600000C4600000C46000015
:1003A0000C4600000C4600000C4600000C46000005
:1003B0000C4600000C4600000C4600000C460000F5
:1003C0000C4600000C4600000C4600000C460000E5
:1003D0000C4600000C4600000C4600000C460000D5
:1003E000FE340000583800000C460000D02B0000FE
:1003F00062410000383100000C4600000C4600004D
:10040000FFFFFF00FFFFFF00FFFFFF00FFFFFF00F8
:10041000FFFFFF00FFFFFF00FFFFFF00FFFFFF00E8
:10042000FFFFFF00FFFFFF00FFFFFF00FFFFFF00D8
:10043000FFFFFF00FFFFFF00FFFFFF00FFFFFF00C8
:100800006FEB200040FE2100000188000000000086
:100810000C000700404E24000100200011000700DA
:10082000000020000000E000020032000000020092
:1008300000000000443C0200000000000040DA001C
:100840000000FE004440A900000020000000E0007D
:100850000300320000002000A00188004440A800EE
:100860000000060091018800800078000000EB0085
:1008700015003700E280400032A0B4009101BA00B8
:10088000E280400032A0B4009102BA00E280400051
:1008900032A0B4000002EB00472BDE00F507B200E7
:1008A000602CE10004003A000059EB008301E900EC
:1008B000FDFF3E00040037006128E1000100320026
:1008C0000082EB00040007001101BA000200E00002
:1008D000E8FF3A00000006003159BA008301E90040
:1008E0000C0032002159BA008301E90008003200EF
:1008F0000400E00003003A00E280400032A0B400AF
:10090000F5FF370011D9BA008301E900FAFF3A0078
:100910008100E800E180400032A0B4000000060041
:10092000889FBE008A9FBE00010578000100E0009C
:100930000400350008003C000000E0002000320008
:100940000500370060001000E080180002003B0046
:1009500001F02C001A0037000004BE006011B8003E
:100960006B0920000982CF00020039000882CF0005
:100970000441B000694252000E00320008003B0002
:1009800082817100610164008904D1000884D30070
:100990008B05E8000442E800F9FF3A000500370043
:1009A0000804440089844C008B05E9000442E900F6
:1009B000FBFF3A00920007000AF0A70001F0A00038
:1009C0004F05BE004F04BE000000060003F0A20069
:1009D000889FBE008A9FBE008C1F7800AE00070073
:1009E000B50033006450E1004F0032006420E100A4
:1009F0005200320003826C0007003B000905D00062
:100A00000306D000820F54000C065D00020039007E
:100A100002003200890178000306780085825500C3
:100A200004003D000003FD008103FD008502EA0093
:100A30008B854200840F720002003B0060001000B2
:100A4000E08018006011B8000005EB007A28E10092
:100A50000A00390006007800C75DDD00F707B20024
:100A6000878075002D003700828171000A017800AF
:100A7000610560008180D1000080D3008502E9001B
:100A8000F9FF3B00060440008784480002003B0059
:100A900060041400E0841C000988A30007003200F1
:100AA0008A81710082817100610164008904D10032
:100AB0000884D3008B05E800170037000978A300ED
:100AC00013003A000B00E000130034008B05E9002E
:100AD0000804440089844C000A4474000978A30087
:100AE0000D003A000B00E000070034008B05E90020
:100AF0000804440089844C0001003A000B002000E7
:100B00000978A300F7FF32000001EB000200370074
:100B1000828171000A017800390007000CF0A700FB
:100B200001F0A0006D0037006420E10002003A00EF
:100B3000838F6C006D0033000801BE000200BE0010
:100B400066003700F4FF2F006B0037001400200010
:100B5000690037006022B800060220000000D000C3
:100B60008180D2000482D2008582D2000000A000E1
:100B70000202520083825A00030031000202420046
:100B800083824A000000A1000603E900F3FF3A0057
:100B9000000006000001BE00720007000470A700FC
:100BA00003F0A10003F8A30013003A006509B100A7
:100BB00010003200090035006928E100020035000C
:100BC000010028000000050000004000818048006E
:100BD0008502E900FCFF3A0000000600F88F4200A1
:100BE000050035008100D1000080D3008502E800B7
:100BF000FCFF3A00000006008000EB00000005004A
:100C000081002000618055000B003D000B0020009A
:100C100061FE2F000100E1001D003400828171009F
:100C2000610164008904D1000884D3000000E80059
:100C3000FAFF3A00710020006100640003007000B8
:100C4000020060000900320061044400E0844C00AE
:100C50000988A500050032008B05E8006808E1005E
:100C600002003A008904D1000884D300F20F20006A
:100C70000258E10005003D00C75DDD00F907B20044
:100C80008980750008007800000006000BF8270036
:100C90008B007800000005000004BE003100070052
:100CA0000003BE000405BE000200BE002D000700C8
:100CB000844F7500000006000200BE006450E10091
:100CC000050036006420E100020036000968A30038
:100CD00001003A000800BE000160A0004F06780045
:100CE0004F05BE004F04BE0000000600F0FF2F00BD
:100CF000F1FF2700F9FF3700889FBE008A9FBE00E2
:100D0000841F7800E4FF07004F00780011003300D3
:100D1000F0FF2F00838F6C0006003B000405650088
:100D20000A00A7000800370009F0A6001000200004
:100D300008003700820F5400838F5C0003003900E5
:100D40001000200001003E000000200009F0A70074
:100D50000000EA004F05BE004F04BE000000E000A6
:100D600000000600C70ADE00F107B200F50FB2006E
:100D700008003200E1CF4200020032000170A00002
:100D800024000500810F70000100320004080500F6
:100D900044000500810F700002003A0014000500B5
:100DA0008502E9000000400081C04800FCFF3B00D4
:100DB0000170A0002400050000A0FE00841F780040
:100DC000851F7800881F78008A1F78004400F8008B
:100DD000080F2000280288000004900010059000F1
:100DE000A000900030019000C00190000300CA00F4
:100DF0000280CA000030CB001A00CD004604C300B8
:100E00000100CA004604C0001E04C0000605C00060
:100E10000100CD0021009800050D7800EABA970086
:100E2000052578004400F9004F0578004F0478004C
:100E3000CF0278004F0278000080FE00000006001C
:100E4000801F78004000B0000008EB004F007800E1
:100E5000801F7800100090000018EB000018EB00D5
:100E60000008EB004F00780000000600686DA80045
:100E7000604380008080FB00216A88004800DE001B
:100E8000306A8800000006000400FA00881F78001D
:100E900041002000B11788008488A90000002200CA
:100EA0003044880070B3270080458800C0A8A9009E
:100EB0008808A9008868A9008888A80088A8A900CF
:100EC0000004EB00584488006844880000A020001B
:100ED00050468800001C22006046880000B02000B8
:100EE000704688000020B0008046880000C82000BE
:100EF000B046880000902100C046880030132300CF
:100F0000F046880000302200004788001047880023
:100F1000E608A900E628A800F00F200090698800E4
:100F200050002000A0698800D0082000B069880027
:100F300020002000C0698800D0698800A2FF24003A
:100F400003002000D2BF9F00E3BF9F0066815700CF
:100F5000E0CD20007D1D0700E0CCBF000080FB003D
:100F6000E0698800DFCCBF000080FB00F0698800EA
:100F700084A8A900E03F2E00B04B880000E02200CA
:100F8000C04B880000002600D04B88007000200075
:100F9000E04B8800F84B8800084C8800184C88000B
:100FA000284C88004F0478000080FA0000000600FA
:100FB000C0508000E10F500026003A00D17280003E
:100FC000301F2000808F5000220036005A2EEF0084
:100FD000F005200080668800DBC2BF000018A30077
:100FE00002003A00E005200080668800DBC2BF00F6
:100FF0000028A30002003A00D0072000D02CB60041
:10100000DBC2BF000038A30002003A00B007200096
:10101000D02CB600F0072000816680008080600040
:10102000511088008488AB000A003A0000042900AF
:10103000301088008600A900ACC0BF0081CFB3008B
:10104000014060000024A000ACE0B7009600A800BA
:101050008488A800000006000000EB00E043880040
:10106000F04388001067800000448800106780000B
:10107000E10F50000400360011678000900320004B
:10108000808F50001000360011678000D0032000D0
:10109000808F50000400360011678000F00D2000A2
:1010A000808F50000800360011678000F00E20008D
:1010B000808F500007003600116780006F004000ED
:1010C000808F500003003E00200020000044880074
:1010D000120037007AC8BF00E24F50000B003A0000
:1010E00011678000F00D2000808F50000B0036004B
:1010F0001167800070004000808F500007003E00A4
:10110000300020000044880004003700E14F500008
:1011100002003A00400020000044880001448000A2
:1011200060FC2F0000804000E30F500005003E00EF
:10113000CACDA900CA2DA900CAADA900CA4DA900EF
:10114000CA8DA900E48F5000AC00320004003E00BC
:10115000E18F50005D003200A3003E000F00370019
:10116000B0032000808F50000A01320004003E00CE
:101170000000E900808F50004F013A00A3003700C3
:10118000C0032000808F5000270132000000E800DB
:10119000808F500048013A003A013700E60CE20027
:1011A0001100320030678000EF0F50000E003E004B
:1011B000306780002167800000004000010040008F
:1011C00001102000810F500007003E007748E20028
:1011D00005003A008000EB00A087200042C0B30069
:1011E000904F11000100320011002000C808DD00FE
:1011F000204480000080A10001007000204488008D
:10120000E60CE20003003A0010002000306788007E
:101210000500370030678000EF0F500002003600F5
:10122000F000200030678800402DEF00316780001B
:10123000006A8000808F50001F0136002544800026
:101240000510B20044D12000F34380000500E00007
:1012500005003200006A800000004000A1AF2F00AE
:1012600001307A0011003700E40CAB0005003200B9
:10127000006A8000000040008000EB0001307A002E
:101280000A003700026A800020678000016A80003F
:101290000000D100010040000000400002014100B8
:1012A00061882000E080780001317A008381E800C5
:1012B000402DEC0031678000006A8000808F500074
:1012C000E2FF3E00F3438800FB0037007AC8BF000E
:1012D00063405000EE4F500003003E000000EB0062
:1012E0007748E2000100320010002000C800DD0055
:1012F000204480000080A10001007000204488008C
:101300007AC8BF00E24F500003003E0030C0B30077
:101310007AE8B70004003700F14F500002003600B1
:1013200010C1B3007AE8B700402DEF00016A8000D9
:101330007AC8BF000080FB000080E900810F5000E8
:10134000DD003600264480000610B20045D12000A2
:1013500027CE20007AC8BF000080FB000082E90091
:10136000F34380000600E00005003200006A8000C0
:1013700000004000A1AF2F0001B07A001300370039
:10138000400DEC000000400060807B000008A300DE
:1013900005003200006A8000000040008000EB0081
:1013A00001B07A0009003700026A8000400DEC00AD
:1013B0000000400060807B000000A10002014100AD
:1013C00061882000E080780001B17A008381E80024
:1013D000402DEC00006A8000800F5200E1FF3E00CB
:1013E000F3438800B400370050552500A0688800FA
:1013F00020002000F0438800AF003700142DEF00DC
:1014000020002000F0438800AB003700CA2DA80060
:10141000CA6DA9007748E2005C003A007848E20013
:101420005A003A0084C8AB0058003200BE0DE200FA
:1014300056003A00CAADA80050678000E40F500083
:101440009D003200556780000500E0004D003A0025
:1014500020678000F00F50004A003A00306780009B
:10146000416780004800DD00010040004402DE00CA
:10147000246D88000004200000005200F1032000C9
:10148000810F50008C003600CBADA900CB4DA900D8
:1014900061688000206780003267800043678000B9
:1014A0000200400003004000808040006168880026
:1014B0008401780000022000800F520010003A00E2
:1014C000E566880050002000D06688008000780023
:1014D0000501780024CE20000180400060007A00E1
:1014E000000141008100E800ED8F5000FAFF3A0052
:1014F000D1668800E2668800020078000C2DB400F6
:1015000052002000110009008281D80001007800FB
:10151000E40F500003003A0040012000606D880095
:101520000200370060012000606D8800226D80009D
:1015300053002000110009000381D8000001780049
:1015400001007800926D88004611DD006D00B90041
:1015500000014100226D88004810DE0030678800DD
:101560000281FB0042678800CAEDA800982DEF00B9
:1015700010002000F06D8800E648A900E668A90088
:101580004D003700506780004B003700CAADA900FE
:10159000490037007748E2000E003A0020678000DB
:1015A000F00F50000B003E00F06D80000000E000E6
:1015B00008003A00CCEDA80031678000516D88002A
:1015C00042678000426D8800306D88006B00070024
:1015D00039003700CCEDA900402DEF0020678000D6
:1015E000016A80000000D100808F50000B003100A4
:1015F00043D12000A2AF2F00006A8000000040000D
:1016000002B07900402DEC0020678000016A800064
:101610000000D100810F5000F7FF3E0020678000DE
:10162000F04388002400370084C8AB001200320069
:101630007748E2000C003A00216780000005200096
:10164000808F500008003A00316780006800500029
:10165000808F500004003A0077005000A068880096
:10166000CA4DA8001400370050052000A06888006B
:10167000CA4DA90010003700A00F2000A068880004
:101680000D0037007748E20006003A00BE0DE20088
:1016900004003A0010032000A0688800CA8DA8004A
:1016A0000300370050052000A0688800CA8DA900FB
:1016B00010002000F043880000000600506D8000FC
:1016C0004800DD00416D8000010040004400DE0064
:1016D000206D880052002000110009000280D8000F
:1016E000906D8800E48F500003003A000001200054
:1016F000006E88000200370010012000006E880094
:10170000236D800052002000110009008281D80062
:101710008001780001007800C619DD006D00B90075
:1017200080814100236D88004818DE003067880002
:101730000380FB00406788000000EB00C06C88005D
:10174000A06D8800CBCDA900CB6DA900CC2DA90040
:10175000B06C8800B0738800CC4DA900CC6DA90096
:10176000C0CC2F008081410020332000808F5100A9
:1017700001003E00CC4DA80000000600CFFF07008E
:1017800020002000F06D880020678000F043880072
:101790007C28EF00CCADA80000000600E648A800B9
:1017A000E668A900C0002000206788008000EB00E8
:1017B000C16C8800B16C8800E16D8800C17388003D
:1017C000016D8800A1CDBF000080FB00306788005C
:1017D000A0CDBF000080FB0040678800CACDA900F3
:1017E000116E8800D0002000006E8800CC0DA9008A
:1017F000316D8800716D8800CBEDA900716E880095
:1018000030002000F06D88001602A800CA6DA90003
:10181000000006007748E20018003A00BE0DE20022
:1018200016003A00618720009140780060C6B3003E
:1018300080CF50000300320000C0E80080CF50008D
:101840000E003A00982DEF00CA6DA900F0072000A5
:1018500030678800800F200040678800200020004B
:10186000F06D8800F0438800A0002000006E880022
:10187000CB0DA800CB2DA8001602A8000000060082
:101880000800FA0070C0B30072E8B7007748E200C1
:1018900036003A0061872000914078000108A300DB
:1018A000040032000000EB007043880075E8B700C8
:1018B0003200370040C6B30080CF50000F003A001E
:1018C00068815700E0FF24000100200000A9BE004D
:1018D00041002000E0CD20001C1B070001CE2000AD
:1018E00091407800C808DD00DFCCBF000080FB001D
:1018F00080804000514788001200370020C6B300A6
:1019000080CF50000F003A00A0FF2400010020000B
:10191000C0BF9F00D1BF9F006881570041002000D9
:10192000E0CD2000091B070001CE20009140780087
:10193000C808DD00DFCCBF000080FB0080804000D5
:101940004147880076C8BF00E00FB20061882000E0
:1019500060807800704388006FC8BF006E48B40094
:101960000040EA0075E8B7000400370050A52A00DF
:1019700070438800E0CFB30075E8B7000080FA003C
:1019800000000600E0C5B3007648E30003003A001B
:1019900020C0B30072E8B7000200370010C0B300E7
:1019A00072E8B7007748E2003E013A0079C8BF000C
:1019B0006EE8B70062872000124178000208A30099
:1019C00043013A00F0C2B300804F5100400136009D
:1019D000E0C5B300804F51003D013E000280FB0096
:1019E000010020002002B1000180B100C3032000EB
:1019F000830F5000E08F580023013E00006001007B
:101A00001B01370020013700190137001E01370084
:101A1000170137001C013700150137001A01370084
:101A20001901370018013700170137001601370078
:101A30001501370014013700630037001201370029
:101A400011013700100137000F0137000E01370078
:101A50000D0137000C0137000B0137000A01370078
:101A600062003700080137008C003700060137009C
:101A700005013700040137008E00370002013700EE
:101A800001013700000137001A003700FE0037005F
:101A900025003700FC00370030003700FA0037001F
:101AA0003C003700F8003700F7003700F600370039
:101AB000F5003700F400370082003700F2003700ED
:101AC00080003700F000370092003700EE0037004A
:101AD000AE003700EC00370080003700EA00370026
:101AE000AE003700E8003700AC003700E6003700F2
:101AF000B80037006146800000F02F0000814000F0
:101B000060438000820F500004003900F00F200075
:101B1000808F5000010036006243880060438000DF
:101B200050468800EA00370051468000021020002D
:101B30000101410060438000820F500004003E001C
:101B4000F0EF2F00808F500001003E0062438800BC
:101B50006143800061468800DD00370081468000D7
:101B6000604380000010B000810F50000600390073
:101B7000F00F2000808F50000300360000F02F008F
:101B80000080400060438800624380007246880005
:101B9000CF00370071468000021020000101410093
:101BA00060438000820F500004003E00F0EF2F00E1
:101BB000808F500001003E00624388006343800034
:101BC00083468800C20037006C08E200C0003A007B
:101BD0000000EB00B0458800602EEF00622EEF00A1
:101BE00090458800A0458800B9003700C1862000D4
:101BF000914078000181FB0002007800000AB200E9
:101C0000B3003A006DC8BF00400CB200B0003A000B
:101C100067016100E50F5100AD003C00E30F51008A
:101C2000AB00320064438000F03723008001620083
:101C300000042000808F510003003A00004680001D
:101C400003006000A20032008180FB00004680009B
:101C50000080FB00808F500005003200E20F510031
:101C600002003400E50F510001003A005E28A80090
:101C7000C0C8AB0004003A00040078000060A10076
:101C8000004688000100370004468800C0A8AB0069
:101C90008F003A00DC22A9008D00370060438000ED
:101CA0000000E0008A00320010468800C0C8A8008A
:101CB0008700370060438000304688005E48A800F7
:101CC0008300370082007800E10FB20060882000B6
:101CD00062438000823078007D00370061438000DD
:101CE00030132300808F500002003600F046880039
:101CF00077003700F0FF2200808F500003003E0085
:101D00000000E800F046880071003700F1468800C6
:101D10006F0037006CC8BF00FC4F50000800320055
:101D2000F84F50000D003600C1C1B3000040EB0079
:101D3000F3020700B1C4B300814F500003003A0022
:101D4000822EEF0049FC070061003700C0862000AA
:101D500083C1B30090CF11005D003E00C1C1B3004C
:101D60000040EB00E6020700B1C4B300814F500011
:101D700003003A00200020001074880001003700A2
:101D8000822EEF0039FC070051003700688DA80053
:101D900060438000106A88004D0037006343800074
:101DA00000302200808F510005003E008200780044
:101DB000E10FB200608820008330780044003700D3
:101DC000E20FB2000130220060882000013178006B
:101DD0003F00370084A8A800402DEF00006A800073
:101DE000E60F500016003E0014C0B30023CE2000C2
:101DF00022D32000006A800000004000E0807900CB
:101E0000006A80000000400060007900808F500070
:101E1000010032000042EB00402DEC00006A80001F
:101E2000E60F5000F3FF3600E1006200C508DD0058
:101E3000204480000050A100010070002044880070
:101E400084A8AB000500320010C3B3006EE8B700F1
:101E5000F0CCB3006FE8B7001D00370050C5B300E9
:101E60006EE8B700B0CAB3006FE8B70018003700DB
:101E700082007800E10FB200608820006243800099
:101E800082307800120037006C08E20010003A003F
:101E9000E20FB2008000EB00608820000131780082
:101EA0000B00370079C8BF000080EA008180EA009B
:101EB0006EE8B700E0C5B3007648E30004003A00DE
:101EC000694050006EE8B700B0CAB3006FE8B700D1
:101ED000000006003600F800809FBE00829FBE0012
:101EE000849FBE00869FBE006228EF0008C2BF002C
:101EF0000048A3002C0032002044800063006000F2
:101F0000E10F50001D003A0007C2BF000048A300C7
:101F1000010032000842A9006AC8BF008080FB00AF
:101F20000128A300090032000118A30005003200B7
:101F30000014A1006AE8B700001080006CE8B70048
:101F40007768B4004EFE0700080037000138A30090
:101F5000050032000034A1006AE8B70000108000DC
:101F600079E8B7007768B40086FE07008448A800C7
:101F70007768EF006AE8EF00B70137008408A9002E
:101F80008428A9008448A9008468A9006AE8EF00B1
:101F90000040EB0072E8B70077E8B70000FC2F00C4
:101FA0000822B600AC01370008C2BF000018A30029
:101FB000BF00320008C2BF000058A300BC003200BE
:101FC00008C2BF000028A300230032008428AB0011
:101FD0002100320021872000914078000108A300F1
:101FE000070032006EC8BF000080FB0010108800A0
:101FF000014078000004A10072E8B700AA00370091
:102000000180FB000018A300070032006FC8BF006A
:102010000080FB0010108800014078000014A1002F
:1020200072E8B700A00037000028A30007003200C4
:1020300075C8BF000080FB001010880001407800C8
:102040000024A10072E8B70097003700F00F2000CD
:10205000101088009400370008C2BF000018A300C9
:102060009100320001108000014178006AC8BF0071
:102070000008A300070032000004A1006AE8B700CE
:102080000100780076E8B700014078007768B40076
:10209000850037008080FB000118A3001B00320080
:1020A0000014A1006AE8B700020078006CE8B700ED
:1020B000024078007768B400E0C5B3007648E300DA
:1020C00006003A0084E8A8000280FB001067880040
:1020D00010C0B3007AE8B7007300370084E8A900A5
:1020E0007A68EF00618720009140780080C6B300D5
:1020F00080CF50000300320000C0E90080CF5000C4
:1021000069003A00C3FD0700670037000128A300FB
:10211000160032000024A1006AE8B700020078002F
:102120006DE8B70084E8AB00060032000280FB00D7
:10213000206788000200780078E8B70020C0B3006C
:102140007AE8B7006DC8BF007768B40011678000F7
:10215000D0032000808F500053003A0084E8AB0089
:1021600051003200BCFB07004F0037000138A300CC
:10217000120032000034A1006AE8B70002007800C3
:1021800079E8B700024078007768B40084E8AB00D3
:102190000700320030C0B3007AE8B7000280FB00CD
:1021A00030678800024078007868B4003E0037004D
:1021B000E62CEF00F3FD07003B003700A38720006B
:1021C00093417800E6CF51001A003E000380FB00E7
:1021D0000281FB000000400021CE200002B0780008
:1021E000608078007768B40084E8AB002200320099
:1021F00011678000B0032000808F500003003A0078
:1022000041C0B30081CF5100080032001167800047
:10221000C0032000808F500017003A00A0872000E4
:1022200031C0B30090CF100013003A008AFB0700C2
:1022300011003700E7CF510008003A001167800015
:10224000F00F2000808F500004003A000240780018
:102250007768B400CBFD0700070037000380FB0060
:102260000281FB000000400021CE200002B0780077
:10227000608078007768B40020678000A187200024
:10228000914078008180FB0066004000808F500004
:10229000040031000180400021CE200060807800E1
:1022A0007868B4007A68EC000782A800EA0037007A
:1022B00008C2BF000018A3000600320008C2BF0019
:1022C0000018A300E400320008C2BF000058A300B9
:1022D000E1003A008468A8006428EF0008C2BF004B
:1022E0000028A30003003A0008C2BF000018A300A2
:1022F000D900320008C2BF000028A300CE0032007F
:102300008428AB0052003200E0C5B3007648E300F9
:1023100004003A0011678000F00F2000808F500009
:1023200022003A0021872000914078000108A30094
:10233000070032006EC8BF000080FB00101088004C
:10234000014078000004A10072E8B700AD0037003A
:102350000180FB000018A300070032006FC8BF0017
:102360000080FB0010108800014078000014A100DC
:1023700072E8B700A30037000028A300070032006E
:1023800075C8BF000080FB00101088000140780075
:102390000024A10072E8B7009A0037008468A90001
:1023A000F00F2000101088009600370011678000A1
:1023B000B0032000808F500004003A00CC2DAB0009
:1023C00002003A007C08E2008E003200E143800007
:1023D000F0438000808F50000700390031882000D2
:1023E000914078008180FB00001020000100500027
:1023F00010108800140037000108A30006003A00FE
:10240000010078000000A10041D120006080780028
:1024100082E8B700060037000100E9000000A100D3
:1024200041D12000608078004800DE0082E8B700DB
:1024300021882000914078000180FB001010880066
:10244000014078008368B4007C28EC006D00370000
:102450008408A8008428A8008448AB0011003A0032
:10246000E0C5B3007648E3000A003A001167800037
:10247000F00F2000808F50000600320011678000AE
:10248000B0032000808F500002003200F2FA0700F3
:10249000030037006A68AB0001003200F8FC070057
:1024A0008448A80000108000228720001241780094
:1024B0000204E00006003A00E0C5B3007648E300FD
:1024C00006003200F00F2000101088004D00370089
:1024D000E0C5B3007648E30004003A0011678000CD
:1024E000F00F2000808F500018003A006EC8BF0027
:1024F0000080FB0010108800024078000004A1005A
:1025000072E8B70084A8AB000600320010C3B30025
:102510006E48E30003003A0084C8A800E688A800DB
:1025200038003700E0C5B3007648E30035003A00D4
:1025300011678000F00F2000808F500031003A00BA
:1025400084C8A900E688A9002E003700526E8000DA
:102550000218A3000F0032000258A3000A00320044
:10256000A00A2000101088000278A3002500320085
:1025700060002000D06D8800CA6DA800CC8DA80036
:10258000CAEDA9001F003700A00F2000101088001E
:102590001C00370011678000B0032000808F5000BE
:1025A00002003A00CCEDAB0016003A00A0688000B3
:1025B00082E8B7008080FB001110880083E8B70034
:1025C00010002000E043880084C8AB000700320000
:1025D0000228A3000500320084C8A900E688A900EB
:1025E00040002000F0708800060037000248A30079
:1025F0000400320010C3B3008248E30001003A0037
:1026000066FC07000000EB001C000700116780005B
:10261000B0032000808F500005003A00606E8000FB
:102620002008B20001082000810F50000A0032008B
:102630000782A800080037000010800077E8B70084
:102640000782A8008408A8008428A9008448A9005B
:102650006AE8EF007E28EF000010800008C2A900A1
:102660008600A9004F03BE004F02BE004F01BE000E
:102670004F00BE003600F900004006000000E000F8
:10268000040032008000EB008100E800808F5000E1
:10269000FDFF390000000600EC02A800E802A900D6
:1026A000EC22A800E822A90020002000F3FF070088
:1026B000EC02A90020002000F0FF0700EC22A90096
:1026C00000000600EC02A900E802A900200020009A
:1026D000EAFF0700EC22A80040002000E7FF070007
:1026E000EC02A80010002000E4FF07000000060034
:1026F000889FBE000004EB008084FB000848DD00DA
:102700000078A30002003200EC02A80001003700AC
:10271000EC02A900E802A900EC22A80010002000A9
:10272000D6FF0700EC22A90010002000D3FF07000D
:102730000804E800E80F5400F0FF3A00E802A8009F
:10274000EC22A800A22E2000124178006100610056
:102750000080EA008180EA00406C8800EC22A90039
:102760004F04BE0000000600881F7800866EEF0050
:10277000E802A8000004EB00EC22A90020002000E1
:10278000BEFF0700EC22A80086CEBF0080404000BC
:102790000100780086EEB700EAC2BF000008A3007F
:1027A00003003200014078000004A00086EEB7006C
:1027B0000804E800E80F5400EFFF3A00EC22A900FB
:1027C00020002000ADFF0700EC02A800E802A900ED
:1027D000EC22A80020002000A8FF0700EC22A9009E
:1027E00086CEBF000080FB004F047800000006008A
:1027F000889FBE008A9FBE008C9FBE008E1F7800FF
:1028000080467800814578000247780003467800CA
:102810008E2DEF000D003700E20F50001500320042
:1028200005003E000000E00008003200E10F50000B
:1028300023003A0008003700E30F50002500320063
:10284000E40F50001E003A001C003700680DA8007D
:1028500091FF07001A00370000CAB30000C046000D
:10286000A3FF0700880DE20015003A008E2DEF004F
:10287000130037000B4078009DFF0700880DE20031
:102880000F003A008E2DEF000D00370008004400C5
:1028900061C520006080780095FF0700880DE20088
:1028A00001003A008E2DEF008904E8000804E800DA
:1028B0008A8F540002003100F4FF370081FF0700C7
:1028C0008E0DEC00706C8800E40F5000D2FF3600D3
:1028D000060037000C85FB000C04E000F8FF320016
:1028E0000E84FB008004EB00E8FF37004F07780000
:1028F0004F06BE004F05BE004F04BE00000006009C
:10290000889FBE008044780001447800902DEF003D
:102910000E003700E20F50001500320005003E00A7
:102920000000E00009003200E10F500022003A00F0
:1029300008003700E40F50001B003200120039007D
:10294000E50F50001C003A001A00370052FF070044
:102950001900370000CAB30000C0440064FF07003C
:10296000880DE20014003A00902DEF0012003700AD
:10297000084078005EFF0700880DE2000E003A0074
:10298000902DEF000C00370043FF070010CAB30082
:1029900000C0440056FF0700880DE20006003A0020
:1029A000902DEF00040037006FFF070086EEB700A0
:1029B0000100370043FF0700900DEC00806C880099
:1029C000E50F5000D3FF360086CEBF000080FB002D
:1029D0004F04BE0000000600881F78000004EB00D2
:1029E000386B8800B1C0B30020C0B300C4FF07003B
:1029F0008080FB0021748800E14F40002A003A00EB
:102A000068CDBF000008A30013003A008001EB006E
:102A100062C520008000EB00E4022000038041003A
:102A200001307900E10F540003003A00EF8F5100AC
:102A300001003A00A46388008301E800F08F510090
:102A4000F6FF3A00C440DD000041EB000240780090
:102A500067FF0700010037000804E9000804E800E8
:102A6000EF0F5400E6FF360068CDBF000008A3005A
:102A7000FDFF3A008000EB0063C520000208200043
:102A80000180400002B079008100E800EF8F500023
:102A9000FBFF3A00814178000041EB008240780062
:102AA00020C0B30052FF070068CDBF006144600042
:102AB000FDFF3A0011C0B30020C0B30090FF070033
:102AC0000080FB00D06A880021C0B300014078007C
:102AD0008BFF07000080FB00806A880031C0B300D4
:102AE00020C0B30086FF07000080FB00206B880039
:102AF00041C0B30020C0B30081FF07000080FB008D
:102B0000506A880051C0B30020C0B3007CFF0700AA
:102B10000080FB00C06A880061C0B30020C0B30021
:102B200077FF07000080FB00606A880071C0B30077
:102B300020C0B30072FF07000080FB00E06A88003D
:102B400081C0B30020C0B3006DFF07000080FB0010
:102B5000F06A880091C0B30020C0B30068FF07008E
:102B60000080FB00006B8800A1C0B30020C0B30050
:102B700063FF07000080FB00106B8800884078002E
:102B800020C0B3005EFF07000080FB00906A880051
:102B9000C1C0B30020C0B30059FF07000080FB0094
:102BA000A06A8800D1C0B30020C0B30054FF070062
:102BB0000080FB00B06A8800E1C0B30020C0B30011
:102BC0004FFF07000080FB00706A88008840780093
:102BD000084078004AFF07006AEDB70011C0B30053
:102BE0000840780046FF07006BEDB70021C0B30036
:102BF0000840780042FF07006CEDB70031C0B30019
:102C0000084078003EFF07006DEDB70041C0B300FB
:102C1000084078003AFF07006EEDB70051C0B300DE
:102C20000840780036FF07006FEDB70061C0B300C1
:102C30000840780032FF070070EDB70071C0B300A4
:102C4000084078002EFF070071EDB70081C0B30087
:102C5000084078002AFF070072EDB70091C0B3006A
:102C60000840780026FF070073EDB700A1C0B3004D
:102C70000840780022FF070074EDB700B1C0B30030
:102C8000084078001EFF070075EDB700C1C0B30013
:102C9000084078001AFF070076EDB700D1C0B300F6
:102CA0000840780016FF070077EDB700E1C0B300D9
:102CB0000840780012FF070078EDB700F1C0B300BC
:102CC000084078000EFF070079EDB70001C1B3009E
:102CD000084078000AFF07007AEDB70011C1B30081
:102CE0000840780006FF07007BEDB7004F0478002E
:102CF00000000600881F780068CDBF0061446000B6
:102D00006F013A00660DE2004700320011C0B300C7
:102D100020C0B300FAFE07000080FB00D06A8800E4
:102D200021C0B30001407800F5FE07000080FB00E1
:102D3000806A880031C0B30020C0B300F0FE0700F5
:102D40000080FB00206B880041C0B30020C0B300AE
:102D5000EBFE07000080FB00506A880051C0B30002
:102D600020C0B300E6FE07000080FB00C06A8800B8
:102D700061C0B30020C0B300E1FE07000080FB008B
:102D8000606A880071C0B30020C0B300DCFE070099
:102D90000080FB00E06A880081C0B30020C0B3005F
:102DA000D7FE07000080FB00F06A880091C0B300E6
:102DB00020C0B300D2FE07000080FB00006B88003B
:102DC000A1C0B30020C0B300CDFE07000080FB000F
:102DD000106B88008840780020C0B300C8FE070050
:102DE0000080FB00906A8800C1C0B30020C0B3001F
:102DF000C3FE07000080FB00A06A8800D1C0B300BA
:102E000020C0B300BEFE07000080FB00B06A88004F
:102E1000E1C0B30020C0B300B9FE07000080FB0092
:102E2000706A8800662DEF00620CAB004000320033
:102E3000406B8000620460003D003A00F1C1B300C5
:102E400008407800AEFE07000081FB000274880095
:102E5000E1C2B300814F50000B003A0081CEB300B5
:102E600008407800A6FE07000080FB00006C880088
:102E700091CEB30008407800A1FE07000080FB005F
:102E8000106C88000B003700F84051000040EB0048
:102E90009BFE07000080FB00006C8800017480002E
:102EA000F7C050000040EB0095FE07000080FB00DB
:102EB000106C8800116C8000C808DD00F80F20003D
:102EC000006C80000800600080804000F16B88008A
:102ED000E1C1B3000040EB0089FE07000080FB0069
:102EE000E06B88002163800010638000C808DD006B
:102EF0000800600080804000216C8800F2FE210004
:102F000082806000F06B800002006000808F5000C3
:102F100006003200406B80006400600004003A004C
:102F2000682DA8004074880001003700622CEF0073
:102F3000416B800066806000810032004074800038
:102F4000E20F50003900320005003E000000E000B2
:102F500009003200E10F500076003A002B003700E4
:102F6000E40F50004F00320046003900E50F5000DA
:102F700070003A005800370091C1B3000040EB00E8
:102F80005FFE0700C16480000080FB00010040007C
:102F9000C0628800A1C1B3000040EB0058FE0700EA
:102FA000C16280000080FB00C808DE000100400014
:102FB000D0628800B1C1B3000040EB0050FE0700B2
:102FC000D16280000080FB00C808DE0001004000E4
:102FD000E062880033C0B30012C0B30091C1B300F7
:102FE0000040EB0002FE0700182EEF00684DAB001A
:102FF000040032006000200040748800684DA90081
:10300000AF003700882EEC00AD0037001300200021
:10301000B36288000041EB00D1C1B30002407800E8
:10302000F3FD0700882EEC00A50037007C0DEC00B6
:10303000B0628800B06280007200200011000900B8
:103040000280D800616C88000100E00001003A00B5
:10305000626C8800636C800083814100936C8800FF
:103060006E801100A06C88000041EB0001E8200098
:103070009140780002407800DDFD0700882EEC00CA
:103080008F003700926C800003E8200093404100DD
:1030900003C1B3000040EB00D5FD0700882EEC0013
:1030A00087003700A36C80000300E00008003200B6
:1030B00021D920009140780070C140000074800048
:1030C00080C04000F0C040000040EB00C8FD070099
:1030D000882EEC007A003700007480007E004000EB
:1030E00000748800F10F2000810F500002003600AC
:1030F000E0022000007488000004EB00986488005F
:103100007C0DEC00A064880001748000B16488002C
:1031100033C0B300E2C1B300D1C1B30008407800AE
:10312000B3FD0700682DA900882EEC001863880005
:1031300063003700600020004074880060003700A2
:103140000148A30016003200C1C1B3000040EB00EB
:10315000EBFD0700B1C4B300814F500007003A00F7
:10316000C086200083C1B30090CF110003003E0051
:10317000200020001074880001003700822EEF002C
:1031800021D420009140780082CEBF00DCFD0700F2
:103190004800DD00E0468800688DA900480037003F
:1031A0000138A3002E003200306A8000D06488000D
:1031B00014748000E20F520013003A00206A80006D
:1031C000EE0F500010003E00C1C1B3000040EB0004
:1031D000CBFD0700B1C4B300814F50001E003A0080
:1031E000206A8000EB0F50001B003200130020000B
:1031F000336B880022C2B3008040780082CEBF00CB
:103200007BFD07001400370013C0B30022C2B300D7
:1032100041D42000914078000440780074FD0700FC
:10322000820EE2000C003A00226A8000F10F510089
:1032300009003E0040022000020040000000400063
:1032400061C52000D364800003B07800D1648000A1
:10325000A0D6200001717800686DA9001800370021
:1032600040758000E10F400014003200517480006E
:103270000100DE000008A3000A003A00818040003F
:1032800040C2B30000C1400023C0B3000040EB00C7
:1032900057FD070010002000517480000100DD0080
:1032A000A82EB7008A0EEC0050748800E80F50007A
:1032B000030036008A2EEF00010037008A2EEF004F
:1032C0004F04780000000600CA0DA900BE2DEF00D3
:1032D00000000600CA0DAB000C003A0000202800D8
:1032E000B0108800B0182000A01088008A40A90003
:1032F000BDC0BF0081CFB300014060005040B300AB
:10330000BDE0B7009A40A800CA0DA8000000060062
:103310003600F800809FBE00829FBE00849FBE00E2
:10332000869FBE00C82DEF00CACDAB0088003A00D2
:10333000C36C8000E28F510003003E00E18F51001A
:103340000C00310003003700E38F510037003A00D2
:103350001200370018E2A900000A2000901088002F
:103360001842E200FBFF350010002000C06C88000E
:10337000B002370018E2A9000301E8008200410012
:1033800020CE200061007800901088001842E200F2
:10339000F8FF3500C26C8800A6023700F16D80008E
:1033A000E68F5000A3023E00100020008100DD00E7
:1033B00001007800C006B20010003A000148A300E6
:1033C00012003A000118A3009A02320001C8B300AB
:1033D00018E2A900606780009010880018C2BF0042
:1033E00001406000FAFF3A0040002000C06C8800F5
:1033F00060002000306E88008E0237001622A80080
:1034000040002000C06C88008A02370018E2A90042
:1034100062688000921088001842E200FBFF3500CD
:1034200040002000C06C880082023700F16D8000EF
:10343000E68F50007F023E00100020008100DD007A
:1034400001007800C006B20032003A000148A30033
:103450003A003A000118A30076023200316E800073
:10346000606D8000808F500011003100638060002B
:1034700002003A000100E800306E8800306E8000E3
:103480008000400023CE200002C8B30018E2A9004B
:10349000618079009010880018C2BF00024060006F
:1034A000FAFF3A00982DEC00C62DEC0061023700BF
:1034B000808F50005F023A000100E800306E880003
:1034C000CBADA8001642A800606D8000F40F50003C
:1034D0000E003A00CB4DA800916D8000F01F200037
:1034E000808F500053023E00403320000100400016
:1034F000206D8800C800DE00316788000080FB0076
:1035000040678800CA6DA8004A023700BE2DEF0050
:103510004802370018E2A900100A20009010880025
:103520001842E200FBFF3500CACDA8000000EB0006
:10353000B06C8800B07388003E023700CBADA900A4
:10354000CB4DA9001642A800BE2DEF00390237006E
:1035500018C2BF000018A3002E01320080108000A6
:1035600074EEB7001822A900B26C8000006E8000D3
:10357000800F5100BD003100F06D8000E20F50005F
:1035800030003A00B47380008401E800B37388000F
:10359000216D8000A0192000808F500002003A00A9
:1035A000E70F51000300360074CEBF000080FB001F
:1035B000B42DB4000308A3000E00320074CEBF0087
:1035C0009EEDB7008480E8006380600023003A002D
:1035D0009FEDB700962DEC00B17388008400780051
:1035E0000100A10040D12000F26C80008230780000
:1035F0001A00370074CEBF009FEDB7000400E90049
:103600000000A10041D12000F26C800002B07800DF
:10361000CB0DAB0005003200EA8F510003003A00E9
:10362000E068800070478800CB0DA900CB2DAB006F
:103630000A003200A268800062478800CB2DA900F2
:1036400006003700F06D8000E50F500003003A00DF
:1036500074CEBF000080FB00B42DB400B26C8000BB
:103660000201E800B26C8800F06D8000E30F5000AA
:103670005D003A00EC0F51003D003E00116E8000ED
:103680007D004000808F500002003A00E60F51009C
:103690000300360074CEBF000080FB00AE2DB400E6
:1036A000116E8000F09F2000808F500069003A006A
:1036B000006E8000EC0F500066003A00B06C800095
:1036C000EC0F500008003A0074CEBF000080FB00F1
:1036D000706E88004800DD00816E800001004000AF
:1036E000704788005B003700EB0F500004003A0081
:1036F00074CEBF000080FB00806E8800550037004C
:10370000E60F500008003A0074CEBF000080FB00B6
:10371000A06E88004800DD00916E8000010040002E
:10372000604788004B003700E50F500004003A0066
:1037300074CEBF000080FB00906E8800450037000B
:10374000E90F500004003A0074CEBF000080FB0077
:10375000D07388003F003700E80F50003D003A006A
:1037600074CEBF000080FB00E07388003900370092
:10377000ED0F510037003A00006E8000ED0F500051
:1037800034003A0074CEBF000080FB00806D8800DA
:10379000106E8000FF0F500004003600116E800094
:1037A000F0032000808F500004003600116E80006E
:1037B000F0072000808F500026003600CC0DA800B6
:1037C000806D8000AE0DB4000080FB0003003A0065
:1037D000CBEDA800306D88001E003700CBEDA900AE
:1037E000A62DEC001B003700F06D8000E60F5000A6
:1037F00018003A0074CEBF000080FB00806D880086
:10380000106E8000FF0F500004003600116E800023
:10381000F0032000808F500004003600116E8000FD
:10382000F0072000808F50000A003600CC0DA80061
:10383000806D8000AE0DB4000080FB0003003A00F4
:10384000CBEDA800306D880002003700CBEDA90059
:10385000A62DEC00B16C8000006E8000808F5000BF
:103860000200310016A2A9001682A800B16C8000E7
:10387000006E8000808F50006E013A00F06D800075
:10388000E20F500060003200F06D8000E30F500046
:103890001F003A00C22DEC00CA0DE2000300350003
:1038A000306D8000E30F50000F003A00A62DEF00AE
:1038B000726D800002007800BC2DB400116E800093
:1038C00000022000808F50004F003600116E8000F3
:1038D00000042000808F50004B003E000200780062
:1038E000782EB40048003700E20F500046003E003A
:1038F000CC0DAB0044003200006E8000ED0F500094
:1039000041003A00CC0DA900C22DED003E00370069
:10391000F06D8000E60F50003B003A00CA0DE20057
:1039200003003500306D8000E30F500030003A0096
:10393000726D800002007800BC2DB400116E800012
:1039400000022000808F500006003600116E8000BB
:1039500000042000808F500002003E00020078002A
:10396000782EB400116E800000A02000808F5000DF
:1039700025003A00D07380004800DD00E17380002C
:1039800001004000C173800081014000C3738800C2
:10399000706E8000F20F20000280B900BC2DB400D0
:1039A000BC0DE2000F003A000300E0000D003A00F9
:1039B000704780000000E0000A003200E10F400084
:1039C00008003200604780000000E000050032007F
:1039D000E10F400003003200E648A800E668A800B6
:1039E00009003700E648A900E668A800060037008D
:1039F000E20F500004003E00CC0DAB00020032008C
:103A0000CC0DA900C22DED0016A2A8001682A800B8
:103A100008013700B16C8000006E8000808F50007C
:103A2000020031001662A800020137001642A80009
:103A3000982DEF00CACDA900F06D8000E30F500073
:103A400003003200F06D8000E60F50005C003A0089
:103A5000106E800003A02000830F500056003E002F
:103A6000106E800052002000110009000280D80072
:103A70000100E00013003A00F06D8000E60F5000F6
:103A800003003A00106E8000830F50000D003A00D2
:103A9000106E800052002000110009000280D80042
:103AA0000100E0001F003A00006E8000ED0F5000A2
:103AB0001C003A00116E800000A02000808F500092
:103AC0001800320030002000F06D8800126E800077
:103AD000146E800053002000110009000381D800FB
:103AE000000178004611DD00110009000382D800B2
:103AF000010078006D00B90000014100026D8800EE
:103B0000A1CDBF000080FB0030678800A0CDBF00C2
:103B10000080FB0040678800CA6DA800AE2DEF0052
:103B200019003700F06D8000E30F500016003A00D6
:103B3000006E8000EC0F500013003A00106E800001
:103B400052002000110009000280D8000000E900A6
:103B5000206E8800216E8000F01F2000808F5000B2
:103B600009003E00206E80004033B000206D8800C8
:103B7000C800DE00316788000080FB0040678800D5
:103B8000CB8DA800CA6DA800106E800052002000E6
:103B9000110009000280D800E48F500003003A00B1
:103BA000C0002000006E8800A2003700D000200076
:103BB000006E88009F003700BE2DEF009D0037008B
:103BC000F06D8000E20F500055003A00CA6DA90068
:103BD000BE2DEF00CBCDA800A62DEC00006E80001E
:103BE000F00F50000E003A00CB6DA800916D8000E0
:103BF000F01F2000808F50008E003E0040332000D8
:103C000001004000206D8800C800DE003167880098
:103C10000080FB0040678800CA6DA800850037005F
:103C2000F10F500083003A00B4CDBF000080FB00CC
:103C30000000E9004F00DE00610060004300DD008D
:103C4000616E80000130A10080807000616E88008C
:103C50006881600003003A00306D8000E30F50007F
:103C6000020032006C806000260032000128A300B0
:103C70000F0032000000EB00F073880042D12000FA
:103C80008081EB00F40F2000800040008330790039
:103C90000008A30001003200843079000000E80031
:103CA000E80F5000F8FF3A00F07388000C0037006E
:103CB0000200E0000A003A00F273880082007800F7
:103CC00042D12000A3AF2F000180400003307900D3
:103CD0008100E800E88F5000FBFF3A00F173880094
:103CE000A2688000121088000782A800CC2DA800CE
:103CF00010002000E0438800A068800083E8B7003F
:103D00004C0037000200E0004A003A00306D8000AD
:103D1000E20F500047003E0098F6070045003700CC
:103D2000F06D8000E50F500041003A00CA6DA90017
:103D30000000EB00F06D8800B44DE20001003A0095
:103D400010C0B300E1006000C308DD00606E8000B9
:103D50000030A10001007000606E880080007800D3
:103D60006801600003003A00306D8000E30F5000EE
:103D7000020032006C806000260032000128A3009F
:103D80000F0032000000EB00F073880042D12000E9
:103D90008081EB00F40F2000800040008330790028
:103DA0000008A30001003200843079000000E80020
:103DB000E80F5000F8FF3A00F07388000C0037005D
:103DC0000200E0000A003A00F273880082007800E6
:103DD00043D12000A2AF2F000180400002B0790043
:103DE0008100E800E88F5000FBFF3A00F173880083
:103DF000A0688000101088000782A800CC2DA800C1
:103E000010002000E0438800A068800083E8B7002D
:103E1000080037000200E00006003A00306D800024
:103E2000E20F500003003E0054F607000100370087
:103E3000CA6DA90082108000126D880018E2A900E6
:103E400018C2A9008A40A9004F03BE004F02BE005D
:103E50004F01BE004F00BE003600F90000400600D2
:103E600000017800D209AB000E003A0023C2BF0067
